:020000040000FA
:100000008316031318280000B1000308B2008316FA
:1000100003131530811D03018312031381000B119B
:10002000AF08031DAF0332088300B10E310E090083
:100030000E309F005730810021308500FF30860050
:1000400080308700243098004030990083120313D9
:1000500080309F0090309800FF3085008600870038
:10006000203084008001840A33300402031D3228CA
:100070000B308700A50005120000051600001030A7
:100080008700A40005120000051600002330870039
:10009000A300051200000516000030308700A20002
:1000A000051200000516000003018100A0308B003E
:1000B0001A08AF08031D6C281730AF000511851012
:1000C00000000000060805158514B0002E02031973
:1000D0006C283008AE004F228C1E592818197E2833
:1000E00098187E288B131A08A00082208316031309
:1000F00057308100831203138B1759281A081812DE
:100100001816592800308A0020080F398207A428C1
:10011000AC28B428BC28C428C62884298629252AC6
:10012000CA2808000800080008000800080000307D
:100130008A002408073982070134023404340A345F
:10014000143428346434C834200E8700A500051206
:100150000000051600000429200E8700A4000512E7
:100160000000051600000429200E8700A3000512D8
:100170000000051600000429200E8700A2000512C9
:1001800000000516000004293322C7283B22211C49
:10019000CE280729200E0139A10004290330870049
:1001A000A500051200000516000005118514053094
:1001B0008700A50005120000051600008C1EF5281A
:1001C0001819F2289818F2281A080E3C031DF52871
:1001D0000B308700A5000512000005160000153041
:1001E0004F2208001A0818121816851EDE28000073
:1001F000851EDE280000851EDE280B308700A50046
:10020000051200000516000006304F2208002808DD
:10021000A6002908A700A60F0E29A70A0515851014
:1002200081309F00831603135F3081008312031314
:100230009C3081000B1101301E299720AF008B17D5
:10024000AF08031D20298B1300005F21A60B2C296A
:10025000A708031D2F295C2926090319A7038C1E53
:10026000542918195129981851291A080E3C031DB0
:1002700054290B308700A500051200000516000068
:1002800080309F0002304F222608A802031CA903D9
:100290002708A90229084F2228084F2203304F229D
:1002A00008001A0818121816851E1D290000851E40
:1002B0001D290000851E1D2980309F00FD281F1567
:1002C00001308700A5000512000005160000851109
:1002D0000000851509308700A500051200000516ED
:1002E00000001F197129831603138601831203135B
:1002F0001E08860000008511000085158316031373
:100300008609831203130800332287293B220B300E
:100310008700A5000512000005160000211C932986
:100320000515851095290511851402304F222708DF
:100330004F2226084F2208308700A5000512000032
:1003400005160000000000000608AA004F22093030
:100350008700A5000512000005160000211C042AD4
:100360000000000008308700A500051200000516F7
:100370000000000000000608AC004F220930870092
:10038000A5000512000005160000042A08308700A9
:10039000A500051200000516000000000000060878
:1003A000AB0009308700A50005120000051600000B
:1003B000211CEE290000000008308700A50005126E
:1003C000000005160000000000000608AD0009301E
:1003D0008700A50005120000051600002B082A0260
:1003E000031DF829211C042A2D082C020319042AB4
:1003F00027084F2226084F222B08AA004F22211C33
:10040000042A2D08AC004F22A60F072AA70A2708A6
:100410002902031C112A031DC629260828020318D5
:10042000C62929084F2228084F222B084F22211CB9
:100430001B2A2D084F220B308700A5000512000053
:100440000516000080304F22080002304F22240E93
:100450004F22230E4F22220E4F22210E093E4F2201
:1004600003304F2208000030A600A700FF30A8008C
:100470007F30A90008004322A9004322A8000030D1
:10048000A600A70008008C1E432A18194B2A9818AA
:100490004B2A1A0808001A0818121816432A83163D
:0E04A0000313981C512A8312031399000800BD
:02400E00323F3F
:00000001FF
